:0300000002007388
:03000300022010C8
:03000B00022020B0
:0300130002203098
:01001B0032B2
:08002300C0D012070ED0D0324C
:03004000020711A3
:030044000202377E
:030050000207198B
:0300540002032084
:0300580002031888
:03005C0002030F8D
:1000700002032C75D00075812F780079401206F6A6
:1000800090038512032C90033B12032C120711B42A
:10009000200280F840F6B43A51120303F8FC120330
:1000A00003F92CFC120303FA2CFC120303FB2CFCB7
:1000B000BB001688828983120303F0A32CFCD8F7B7
:1000C0001203032C701502008CBB010F1203032CCA
:1000D00070099003B412032C0200869003CB120324
:1000E0002C120711B451FA020086B45303020086A1
:1000F000120719B46203020086B44203020086B4F8
:100100006303020086B46D1D12022888828983125F
:100110000218FAE01200587420120050120050A386
:10012000DAF1020086B44D1D1202288882898312FA
:100130000218FA120218F07420120050120050A394
:10014000DAF1020086B4720B120218F8E6120058B7
:10015000020086B4520B120218F8120218F60200BE
:1001600086B4781A12022820D56375812F7486C050
:10017000E07400C0E0C000C001D2D3D2D422B45891
:10018000030201CDB47A1890037412032C120711E4
:10019000B47903020073B45903020073020086B4F9
:1001A0005A1990037412032C120711B479028006B5
:1001B000B4590575870280FE020086B43F0F900394
:1001C0008512032C90043A12032C020086900340FF
:1001D00012032C020086C2D3C2D4C2D5120040B48E
:1001E000300612005024D022402BB4390280F34054
:1001F000F1B4410612005024C9224019B4460280CD
:10020000F340F1B4610612005024A9224007B466FD
:100210000280F340F1D2D5221201DA20D509C4FEC2
:100220001201DA20D5014E2212021820D508F91247
:10023000021820D501F822C0F080087408120719AE
:10024000D5F0F8B80406E9120318800CB80306E9E3
:100250001203208003B80206EA1203188004EA128F
:1002600003207408120719120711B4270AEAF912B9
:100270000711FA88F080C9B42B0974012AFAE4390D
:10028000F980F0B42D0BD3EA9400FAE99400F980D8
:10029000E2B40813E9C4F5F053F0F0540FF9EAC4DE
:1002A000540F45F0FA80CCB4301724D08AF053F0C4
:1002B000F0C453020F4AC4FAE9540F45F0C4F98060
:1002C000B24027B4390280E240E0B4410424C9803E
:1002D000DB4017B4460280F540F3B4610424A980E2
:1002E000CB4007B4660280F540F3C0E0EA12032079
:1002F000D0E0D0F022120711B4410324C92250FBF0
:1003000024D0221202F5C4F5F01202F545F022C005
:10031000E0E5F0120318D0E0C0E0C4120320D0E002
:10032000540F2490D43440D412071922C0E0E4932F
:10033000A3600512071980F6D0E0220D0A3E2000C6
:100340000D0A5374757069642068756D616E2120A3
:100350002054797065203F20666F722068656C704C
:100360002E000D0A436F6D6D616E642061626F72C5
:10037000746564000D0A41726520796F752073758C
:1003800072653F20000D0A4D6F6E69746F722032E6
:100390002E3020286329203139393720556E69766F
:1003A000657273697479206F6620576973636F6E25
:1003B00073696E000D0A446F776E6C6F6164207311
:1003C00075636365737366756C2E000D0A446F77F1
:1003D0006E6C6F6164206572726F722E2020507295
:1003E000657373205120746F20726573756D652E6F
:1003F00020000D0A436F6465206164647265737345
:100400003A20000D0A4D656D6F7279206164647247
:100410006573733A20000D0A5265676973746572DB
:1004200020616464726573733A20000D0A546F2072
:10043000616464726573733A20000D0A205E422085
:1004400020427265616B2070726F6772616D0D0A78
:10045000202062202041646420627265616B706FAD
:10046000696E740D0A202042202045646974206260
:100470007265616B706F696E74730D0A2020632062
:10048000205669657720636F6465206D656D6F72B6
:10049000790D0A20206D20205669657720657874D3
:1004A00065726E616C206D656D6F72790D0A20202A
:1004B0004D2020456469742065787465726E616CA6
:1004C000206D656D6F72790D0A20207220205669AB
:1004D0006577207265676973746572730D0A2020F1
:1004E000522020456469742072656769737465726F
:1004F000730D0A2020782020436F6E74696E756535
:1005000020657865637574696F6E0D0A2020582028
:100510002053696E676C652D73746570206578650E
:10052000637574696F6E0D0A20207A20205265620F
:100530006F6F740D0A20205A202048616C740D0AD8
:1005400020203F202053686F7720746869732068EB
:10055000656C702073637265656E0D0A546F20645C
:100560006F776E6C6F6164206120686578206669C2
:100570006C652C206A7573742073656E64206974D1
:100580002E000D0A50726F6772616D206578697474
:100590006564000D0A0A4D656D6F727920726F7582
:1005A00074696E6520322E30202863292031393954
:1005B0003720556E6976657273697479206F66208D
:1005C000576973636F6E73696E002020302D394157
:1005D0002D46202048657861646563696D616C20F3
:1005E00076616C75650D0A202027202020202020B0
:1005F00020456E74657220415343494920746578E3
:10060000740D0A20202B20202020202020496E63FA
:1006100072656D656E7420627974650D0A20202DF7
:100620002020202020202044656372656D656E7453
:1006300020627974650D0A20205370616365202063
:1006400020536B697020746F206E65787420627916
:1006500074650D0A2020456E746572202020536B4E
:10066000697020746F206E657874206C696E650DFA
:100670000A202072202020202020205265646973E7
:10068000706C6179206C696E650D0A20206D2020E8
:100690002020202020536574206E6577206D656DC5
:1006A0006F727920616464726573730D0A20203F54
:1006B00020202020202020446973706C61792074F0
:1006C0006869732068656C70206D65737361676518
:1006D0000D0A2020712020202020202051756974CF
:1006E0003B2072657475726E20746F206D6F6E6939
:1006F000746F720D0A0075878075A80075B8007553
:100700008800758922758DFF759852D28E22C2D7C6
:10071000223098FDC298E599223099FDC299F59949
:0107200022B6
:00000001FF
